:020000040000FA
:0400000004EF00F019
:08000800FF0E926E936A946AE8
:1000100092EC00F07AEC00F0C20E12EC01F077ECFA
:1000200000F0026A810E39EC00F0200EB2EC00F014
:10003000010E026E890E39EC00F074EC00F0020E35
:10004000026E910E39EC00F02C0EB2EC00F0990E1D
:1000500045EC00F0200EB2EC00F0050E026EA10E91
:1000600039EC00F0010E16EC01F00FEF00F037EF65
:1000700000F0036E025060EC00F0B2EC00F03A0EBB
:10008000B2EC00F0035045EF00F0046E0450076E30
:10009000EAEC00F00850056E0950066E0550030B9F
:1000A00060EC00F0B2EC00F006380F0B60EC00F0F2
:1000B000B2EC00F006500F0B60EC00F0B2EF00F075
:1000C000086E0A0E085CD8B06CEF00F00850300FD4
:1000D00073EF00F073EF00F00850410F096E0A0E45
:1000E000095C73EF00F01200A80EC0EF00F0800E64
:1000F000C0EF00F0080EC0EC00F0010EC0EC00F004
:10010000C80E44EC01F0020EC0EC00F0C80E44EC46
:1001100001F0060EC0EC00F00C0EC0EC00F0C80EB2
:1001200044EF01F0DBEC00F00A0E1EEC01F08B9ABC
:100130005EEC01F0030ECEEC00F0320E44EC01F068
:10014000030ECEEC00F0320E44EC01F0030ECEECC8
:1001500000F0320E44EC01F0320EC0EC00F0280E3C
:10016000C0EF00F0076E8B8A5EEC01F007380F0BD2
:10017000CEEC00F00750CEEC00F0BFEF00F0120024
:10018000026E8B9A5EEC01F002380F0BCEEC00F0A1
:100190000250CEEC00F0010E26EF01F0086E8B88C5
:1001A0005FEC01F0085060EC01F08B985FEC01F01F
:1001B000010E26EF01F0000E60EC01F08B985FEC71
:1001C00001F08B9A5EEC01F0000E69EC01F094985E
:1001D000949A1200096EC2B0F2EF00F0C280010ED4
:1001E00016EC01F0075004EC01F002EC01F0FEEC1B
:1001F00000F0C450086EC350096E1200C2B4FEEF86
:1002000000F01200C28412000A6E0A50C26E0A5038
:10021000015CD8B40FEF01F0010E1EEC01F00A50A2
:10022000016E1200026E0250C16E12000A6E0A5078
:100230000C6E640E0D6E0A0E2EEF01F00B6E0B505D
:100240000C6E640E0D6E010E2EEF01F0096E09505A
:100250000C6E0A0E0D6E010E2EEF01F00E6EFF0EEB
:100260000F6E0D50116E0C50106EEF0E0F24D8B0A3
:1002700036EF01F0102E35EF01F0112E33EF01F0C3
:100280000E2E31EF01F01200026E0250036E035287
:10029000D8B451EF01F00A0E52EC01F0030647EF1B
:1002A00001F01200046EFF0E056E066A045005246C
:1002B000D8A0000C062458EF01F012001200120022
:1002C000096E09500F0B0A6E8B50F00B0A108B6EE3
:1002D0001200026E02500F0B036E9450F00B0310CD
:0402E000946E120006
:0200000400F00A
:020000040030CA
:0E00000000260E0E00008000F0C00FE00F4042
:00000001FF
